:100000000C9446000C9465000C9465000C946500FB
:100010000C9465000C9465000C9465000C946500CC
:100020000C9465000C9465000C9465000C946500BC
:100030000C9465000C9465000C9465000C946500AC
:100040000C9465000C9465000C9465000C9465009C
:100050000C9465000C9465000C9465000C9465008C
:100060000C9465000C9465000C9465000C9465007C
:100070000C9465000C9465000C9465000C9465006C
:100080000C9465000C9465000C94650011241FBE4F
:10009000CFEFD0E1DEBFCDBF11E0A0E0B1E0E8EBF3
:1000A000F1E000E00BBF02C007900D92A030B10755
:1000B000D9F711E0A0E0B1E001C01D92A030B10776
:1000C000E1F70E9495000C94DB000C940000CF93A4
:1000D000DF93CDB7DEB7EBE3F0E01082EAE3F0E0C8
:1000E00080E48083E8E3F0E01082E7E3F0E0108250
:1000F000E5E3F0E01082E4E3F0E01082E2E3F0E018
:100100001082E1E3F0E01082E3E2F0E080E280833D
:10011000E2E2F0E080E38083E2E6F0E01082E1E6F4
:10012000F0E01082DF91CF910895CF93DF93CDB7A8
:10013000DEB722970FB6F894DEBF0FBECDBF0E9488
:10014000670000C0E9E3F0E080819927817090703A
:100150000097C1F7A3E2B0E0E3E2F0E08081982FDE
:100160008FED892380618C9384EF91E09A8389835A
:1001700005C089819A8101979A83898389819A81AF
:100180000097B9F7A3E2B0E0E3E2F0E08081982FB6
:1001900090628FEE89238C9384EF91E09A83898318
:1001A00005C089819A8101979A83898389819A817F
:0801B0000097B9F7C7CFFFCF9C
:00000001FF
